:020000040000FA
:06000000CA3001303A286D
:08000800A000030EA100831209
:100010008B1C32288B1031181428B11C3228643004
:10002000010203183128182800001628172818285C
:1000300019281A281B281C281D281E281F283110A3
:10004000B114A810031005190314AA0DA90DA80DC9
:10005000B00B322831152A08AF002908AE00280855
:10006000AD00B11081010B11210E8300A00E200EF6
:02007000090085
:0C007400203084008001840A80300402E7
:10008000031C3C281230B000F02183160C3085058B
:1000900087018312850187010730990000309A009B
:1000A000103083168E008312603083168F00831207
:1000B0000030831691009F008312C83083168100A0
:1000C000831231309000003083168C008312103080
:1000D0008B00831600309B001C141A088312BC008E
:1000E000851DE822831610309B001C141A08831209
:1000F000BD00831630309B001C141A088312DE00EA
:10010000CF2281018E018F010B118B100B108C01FE
:100110008B1798203119AE20B30B96280310851940
:100120000314B90DF0303902031954212E23892804
:100130006400311808000B1D08000B11B1103114B8
:100140001230B000051DA928321483160113831242
:100150000800321083160117831208003111013094
:10016000B7008B132030370783169B001C141A0826
:100170008312A400A500C030A506103037078316EF
:100180009B001C141A088312A30000303707831643
:100190009B001C141A088312A2008B17321CD6284D
:1001A00022090339A200A309A409A50922082D02E6
:1001B000031D4E2923082E02031D4E2924082F0259
:1001C000031D4E2901303702031DEB283D18EB2893
:1001D0003D143E14FD2102303702031DF428BD18E2
:1001E000F428BD143E140C2203303702031DFD28F1
:1001F0003D19FD283D153E14182204303702031D19
:100200000629BD190629BD153E14242205303702E2
:10021000031D0F293D1A0F293D163E1433220630C7
:100220003702031D1829BD1A1829BD163E14422293
:1002300007303702031D21293D1B21293D173E149C
:10024000512208303702031D2A29BD1B2A29BD1758
:100250003E145C2209303702031D33295E1833290E
:100260005E143E1467220A303702031D3C29DE1853
:100270003C29DE143E1472220B303702031D45293F
:100280005E1945295E153E147D220C303702031D90
:100290004E29DE194E29DE153E148822B70A0D308C
:1002A000370203180800B1280130B600B300B400CB
:1002B000B500B70085018701B1139820B30B9C29C5
:1002C000031085190314B90DF03039020319C3293D
:1002D000B40B9C29013037020319932202303702F4
:1002E000031998220330370203199D220430370284
:1002F0000319A222053037020319A722063037025C
:100300000319AC22073037020319B1220830370233
:100310000319B622093037020319BB220A3037020B
:100320000319C0220B3037020319C5220C303702E3
:100330000319CA229630B400311D5D293111321CD7
:10034000A6292D090339AD00AE09AF092F1CB11341
:100350002F1C5D29B11B5D292E185D29B1178B1348
:1003600020303707BB002F08BA00DB2110303707D9
:10037000BB002E08BA00DB2100303707BB002D0878
:10038000BA00DB218B1785018701B70AB6010D3052
:100390003702031C5D29CF2208003E1C08003E10D6
:1003A0001030BB003D08BA00DB213030BB005E08D6
:1003B000BA00DB2108008B133A0883161C159A003B
:1003C00083123B0883169B0055309D00AA309D0088
:1003D0009C1464009C18E9291C1183128B170800D7
:1003E000FF30C800CA15CB15CC15CD15CE15CF15CD
:1003F000D015D115D215D3150800C130BD05FF3079
:10040000DE051130C405C0000030C200C600BC18B3
:100410005F14BC18DF140800C230BD05FF30DE05D4
:100420000230C405C0000030C200C6005F100800E2
:10043000C430BD05FF30DE050630C405C000003005
:10044000C200C6005F100800C830BD05FF30DE05E1
:100450001830C405C0000030C200C600BC185F14CC
:10046000BC18DF140800D030BD05FF30DE05303089
:10047000C405C0000030C200C600BC185F14BC1820
:10048000DF140800E030BD05FF30DE053030C40564
:10049000C0002030C200C600BC185F14BC18DF14B6
:1004A00008007F30BD05C030DE05C030C505C10085
:1004B0000030C300C7000800BF30BD05C030DE05F6
:1004C0003030C505C1000030C300C70008003F3010
:1004D000BD05C130DE059030C505C1000030C30048
:1004E000C70008003F30BD05C230DE05C030C5057D
:1004F000C1000030C300C70008003F30BD05C43054
:10050000DE05C030C505C1000030C300C7000800CB
:100510003F30BD05C830DE05C030C505C100003024
:10052000C300C700080010308506023087060800A7
:10053000203085060030870608002130850600300F
:100540008706080002308506023087060800003062
:1005500085060630870608000030850606308706C7
:10056000080000308706183087060800003085062E
:10057000213087060800003085060930870608000C
:1005800000308706183087060800003087061830CC
:1005900087060800003087061830870608003D18D7
:1005A000FD21BD180C223D191822BD1924223D1A27
:1005B0003322BD1A42223D1B5122BD1B5C225E1814
:1005C0006722DE1872225E197D22DE198822080059
:1005D000B601B301B4013C1CF02ABC01BC14F22AE0
:1005E000BC013C143C08B6006400F62AF72AF82A3D
:1005F000F92AFA2AFF30B41B8500B41F8501B30B1A
:10060000F42AB40BF42A0310B60CB608031DF42A1E
:100610000030BB003C08BA00DB21080005125C1862
:100620000516DC1C8512DC1885165C1D05105C198E
:100630000514DC1D8510DC1985145C1E87105C1AFE
:100640008714DC1E0711DC1A07155C1F07105C1BE2
:100650000714DC1F8712DC1B871608008F0803199C
:1006600008008F0178308E00C80F602DC80A441C26
:100670005E2B461C4F2BCA1C402BCA014A156C2B03
:100680004A1D452BCA01CA156C2BCA1D4A2BCA012B
:100690004A166C2B4A1E6C2BCA01CA146C2B4A1DBD
:1006A000542BCA014A166C2BCA1D592BCA014A1673
:1006B0006C2B4A1E6C2BCA01CA146C2BCA1C632BF0
:1006C000CA014A156C2B4A1D682BCA01CA156C2B2E
:1006D0004A1E6C2BCA014A15C41C932BC61C842BC2
:1006E000CB1C752BCB014B15A12B4B1D7A2BCB01B2
:1006F000CB15A12BCB1D7F2BCB014B16A12B4B1E5A
:10070000A12BCB01CB14A12B4B1D892BCB014B165D
:10071000A12BCB1D8E2BCB014B16A12B4B1EA12B3E
:10072000CB01CB14A12BCB1C982BCB014B15A12BB0
:100730004B1D9D2BCB01CB15A12B4B1EA12BCB0110
:100740004B15441DC82B461DB92BCC1CAA2BCC0124
:100750004C15D62B4C1DAF2BCC01CC15D62BCC1D5C
:10076000B42BCC014C16D62B4C1ED62BCC01CC1462
:10077000D62B4C1DBE2BCC014C16D62BCC1DC32B1F
:10078000CC014C16D62B4C1ED62BCC01CC14D62B20
:10079000CC1CCD2BCC014C15D62B4C1DD22BCC0117
:1007A000CC15D62B4C1ED62BCC014C15C41DFE2BC4
:1007B000C61DEF2BCD1CE02BCD014D155F130C2C6E
:1007C0004D1DE52BCD01CD150C2CCD1DEA2BCD01FA
:1007D0004D160C2C4D1E0C2CCD01CD140C2C4D1D8A
:1007E000F42BCD014D160C2CCD1DF92BCD014D1642
:1007F0000C2C4D1E0C2CCD01CD140C2CCD1C032C1F
:10080000CD014D150C2C4D1D082CCD01CD150C2CFA
:100810004D1E0C2CCD014D155F1B352C441E352C67
:10082000461E262CCE1C172CCE014E15432C4E1DD9
:100830001C2CCE01CE15432CCE1D212CCE014E16E4
:10084000432C4E1E432CCE01CE14432C4E1D2B2C7C
:10085000CE014E16432CCE1D302CCE014E16432C0D
:100860004E1E432CCE01CE14432CCE1C3A2CCE016E
:100870004E15432C4E1D3F2CCE01CE15432C4E1E43
:10088000432CCE014E15C41E6A2CC61E5B2CCF1CF9
:100890004C2CCF014F15782C4F1D512CCF01CF156B
:1008A000782CCF1D562CCF014F16782C4F1E782C4C
:1008B000CF01CF14782C4F1D602CCF014F16782C10
:1008C000CF1D652CCF014F16782C4F1E782CCF01F1
:1008D000CF14782CCF1C6F2CCF014F15782C4F1DC7
:1008E000742CCF01CF15782C4F1E782CCF014F15CB
:1008F000DF18A12C451EA12C471E922CD01C832C46
:10090000D0015015AF2C501D882CD001D015AF2C24
:10091000D01D8D2CD0015016AF2C501EAF2CD00105
:10092000D014AF2C501D972CD0015016AF2CD01DD9
:100930009C2CD0015016AF2C501EAF2CD001D014DF
:10094000AF2CD01CA62CD0015015AF2C501DAB2CB9
:10095000D001D015AF2C501EAF2CD0015015DF1890
:10096000D82CC51ED82CC71EC92CD11CBA2CD1011D
:100970005115E62C511DBF2CD101D115E62CD11DEE
:10098000C42CD1015116E62C511EE62CD101D114F4
:10099000E62C511DCE2CD1015116E62CD11DD32CA5
:1009A000D1015116E62C511EE62CD101D114E62CB2
:1009B000D11CDD2CD1015115E62C511DE22CD101A9
:1009C000D115E62C511EE62CD1015115DF18102D42
:1009D000451F102D471F012DD21CF22CD20152159C
:1009E000DF131E2D521DF72CD201D2151E2DD21D44
:1009F000FC2CD20152161E2D521E1E2DD201D214D5
:100A00001E2D521D062DD20152161E2DD21D0B2D4C
:100A1000D20152161E2D521E1E2DD201D2141E2D91
:100A2000D21C152DD20152151E2D521D1A2DD20188
:100A3000D2151E2D521E1E2DD2015215DF18492D22
:100A4000DF1B492DC51F492DC71F3A2DD31C2B2D48
:100A5000D3015315572D531D302DD301D315572DC9
:100A6000D31D352DD3015316572D531E572DD301AA
:100A7000D314572D531D3F2DD3015316572DD31D7E
:100A8000442DD3015316572D531E572DD301D31484
:100A9000572DD31C4E2DD3015315572D531D532DB8
:100AA000D301D315572D531E572DD3015315CD21E7
:100AB0004008C4004108C5005F18DF145F1CDF1048
:100AC0004808C9000C304A05031D05120C304B05BF
:100AD000031D85120C304C05031D05100C304D050F
:100AE000031D85100C304E05031D87100C304F057B
:100AF000031D07110C305005031D07100C30510564
:100B0000031D87120C305205031D07120C305305CC
:100B1000031D871149080E020318BA2D12304A0529
:100B2000031D051612304B05031D851612304C05AA
:100B3000031D051412304D05031D851412304E059A
:100B4000031D871412304F05031D07151230500581
:100B5000031D071412305105031D8716123052056C
:100B6000031D071612305305031D8715FF30480279
:100B7000031908008F08031D0800982049080E0279
:100B8000031CBA2D18304A05031D051206304A050C
:100B9000031D051618304B05031D851206304B0545
:100BA000031D851618304C05031D051006304C0535
:100BB000031D051418304D05031D851006304D0525
:100BC000031D851418304E05031D871006304E0591
:100BD000031D871418304F05031D071106304F05FC
:100BE000031D071518305005031D0710063050056A
:100BF000031D071418305105031D871206305105D7
:100C0000031D871618305205031D071206305205C2
:100C1000031D071618305305031D871106305305B1
:060C2000031D871508000A
:084000000200030004000100AE
:02400E00CC33B1
:10420000010003000300030003000200020002009B
:104210000200000000000000000003000300FF0097
:10422000020000000000000000000000000000008C
:104230000000C000C000C000C000C000C000FF00FF
:10424000FF00C300F300CF00FF00C300F300CF0066
:10425000FF00C300F300CF00FF00C300F300FF0026
:104260000100FF00FF00FF00FF00FF00FF00FF0054
:10427000FF00FF00FF00FF00FF00FF00FF00FF0046
:10428000FF00FF00FF00FF00FF00FF00FF00FF0036
:10429000FF00FF00FF00FF00FF00FF00FF00FF0026
:1042A000FF00FF00FF00FF00FF00FF00FF00FF0016
:1042B000FF00FF00FF00FF00FF00FF00FF00FF0006
:1042C000FF00FF00FF00FF00FF00FF00FF00FF00F6
:1042D000FF00FF00FF00FF00FF00FF00FF00FF00E6
:1042E000FF00FF00FF00FF00FF00FF00FF00FF00D6
:1042F000FF00FF00FF00FF00FF00FF00FF00AA001B
:00000001FF
